:100000003BC0A0C154C053C052C051C050C04FC02B
:100010004EC04DC04CC04BC04AC049C048C047C08C
:1000200046C045C044C00902120001010080190900
:10003000040000000000000012011001FF00000891
:10004000C016DC050401010200010E035500530037
:1000500042006100730070001C0377007700770096
:100060002E00660069007300630068006C002E00BB
:10007000640065000403090411241FBECFE5D4E029
:10008000DEBFCDBF10E0A0E6B0E0E2ECF1E102C0DF
:1000900005900D92A236B107D9F710E0A2E6B0E0C4
:1000A00001C01D92AC3AB107E1F778D888C8A8CF53
:1000B000CF93DF9360918800635067FD13C08091F8
:1000C0008500CCE0D0E0C81BD109C457DF4F809138
:1000D00084008D3209F457C08091620087FD9BC077
:1000E000109288008091600084FF40C060916100A0
:1000F0006F3F09F43BC0693008F46FC068506093EB
:1001000061008091780098E889278093780068E002
:100110008091620087FD1DC040918600509187004C
:1001200086FF70C0FA01862FA9E7B0E094919D93F5
:1001300031968150D9F7262F215030E02F5F3F4F65
:10014000240F351F3093870020938600C62FCC5F85
:100150004FC089E790E0EBD6682F893008F4A1C042
:100160008FEF80936100CEE1C093600094E186B38D
:10017000837031F49150D9F7109289001092830066
:10018000DF91CF910895683009F0AACF83EC809376
:1001900078008AE580936000109262008881807602
:1001A00009F043C09A81109281008981811147C072
:1001B0001092820021E830E082E0309387002093A3
:1001C00086008F3FA9F19F81911104C09E819817ED
:1001D00008F4892F8093610083CF10926100809191
:1001E000780098E8892780937800611191CFC4E066
:1001F00089E790E0A3D0CC3009F4B6CF8FEF80939D
:100200006100B2CFDA01862FE9E7F0E09D9191938A
:100210008150E1F790CFCE01F7D68F3FF1F08823E0
:1002200009F45ECF109261005BCFCE01DBD4C9CF61
:10023000988197FD16C090E890936200CBCF8530EF
:1002400091F0863001F18830D1F0893091F021E8C9
:1002500030E08A3021F180E0B0CF8EE18093600001
:100260003FCF8E81E8CF9093890021E830E080E095
:10027000A4CF90938B0021E830E080E09ECF2BE864
:1002800030E081E09ACF8B81813001F18230B1F092
:10029000833051F080E090E49093620092CF81E04F
:1002A0008CCFC82FCC5FA4CF911118C084E790E009
:1002B000909387008093860084E0EDCF86E290E003
:1002C000909387008093860082E1E5CF88E390E0F9
:1002D000909387008093860082E1DDCF913051F0CA
:1002E0009230C1F68AE490E0909387008093860074
:1002F0008EE0D1CF88E590E09093870080938600D0
:100300008CE1C9CF85B7836085BF8BB780648BBF15
:100310000895A82FB92F80E090E041E050EA609561
:1003200030E009C02D9182279795879510F084279A
:100330009527305EC8F36F5FA8F30895EADF8D93C9
:100340009D930895CF93CFB7CF93C395B09BE9F713
:10035000B09B09C0B09B07C0B09B05C0B09B03C059
:10036000B09B01C0A1C0DF93C0918500DD27C457B9
:10037000DF4FB09B02C0DF91EBCF2F930F931F9302
:1003800006B32FEF00FB20F94F933F9316B34FEFC7
:10039000012700FB21F93BE031C04E7F012F16B34E
:1003A000216028C0102F4D7F2260000006B329C0B5
:1003B0004B7F2460012F000016B32BC016B3477F7C
:1003C00028602AC04F7E06B320612CC04F7D16B333
:1003D00020622FC04F7B06B3206432C0422706B391
:1003E00049934FEF0000102710FB20F916B313704C
:1003F000C9F1297F91F2012700FB21F906B3237F80
:1004000089F2315058F1102710FB22F916B3277EDC
:1004100079F2012700FB23F92F7C81F206B3102724
:1004200010FB24F92F7971F200C016B3012700FBED
:1004300025F92F7359F200C006B3102710FB26F9D7
:10044000223040F200C016B3012700FB27F9243008
:1004500028F64F77206816B30000F9CF10E41ABFD2
:10046000002717C03B503195C31BD04010E41ABF82
:100470000881033CE9F00B34D9F020918300198105
:10048000110F1213EDCF093641F10D3211F0013E7B
:1004900039F700938A003F914F911F910F912F914F
:1004A000DF91CAB7C6FD51CFCF91CFBFCF9118957D
:1004B00020918A00222379F310918800112311F5ED
:1004C000343012F13093880020938400109185001D
:1004D0003BE0311B3093850017C00091880001304C
:1004E0008CF40AE53091600034FD10C00093600088
:1004F000C8E7D0E00FC02795A8F45150A9F4220F07
:100500000000F9CF4AE503C042ED01C0432FC4E12A
:10051000D0E032E017B31360C09A17BB08B320E4F1
:1005200013E05F93012756E008BB279520F4515054
:1005300021F4220FF9CF012756E000003B5A08BBF7
:10054000D0F2279528F4515029F4220F0000F9CF5A
:10055000012756E0279508BB20F4515021F4220FC3
:10056000F9CF012756E02991332308BB21F60C7FF0
:1005700010918900110FC651D04008BB11F01093A3
:10058000830010E41ABF016017B31C7F402F4C7F1B
:100590005F9100C000C008BB17BB48BB7CCF682F71
:1005A00058E080E07091A8002091A70067FD1EC070
:1005B000C398660F880FB4998F5FC59A32B7472FDB
:1005C000415030F092B7931B9217E0F34150D0F7AF
:1005D000C59832B7472F415030F092B7931B92170E
:1005E000E0F34150D0F7515009F70895C39AE1CF95
:1005F0008FB9779BFECF8FB1089521E196958795AE
:10060000779567952A95D1F72091A6002617D9F0FE
:100610006093A600E091A300F091A4008DE40995F9
:10062000E091A300F091A40080E00995E091A3007F
:10063000F091A4008091A6000995E091A300F091AB
:10064000A40080E0099408958091A5008DB980915F
:10065000A2008EB908958823C1F0883008F042C006
:100660002FEC32E03093A4002093A30091E090930C
:10067000A800843039F1D8F0863049F158F187303C
:10068000D1F483E08093A700089588EF92E09093DF
:10069000A4008093A30081E08093A7008093A8002A
:1006A00082E58093A50081E08093A20008958230C6
:1006B00069F0833099F080E68093A70082E0809310
:1006C000A800089588E18093A700089580E68093AC
:1006D000A70008958CE08093A700089580E380939D
:1006E000A700089528EF32E03093A4002093A300E0
:1006F0001092A20091E09093A7009093A8008930F7
:1007000039F050F4883061F683E58093A5000895B0
:1007100082E58093A50008958B3049F08C3009F074
:10072000BFCF81E58093A5009093A200089581E555
:100730008093A500089522B73091A8009091A7005A
:10074000315030F082B7821B8917E0F33150D0F777
:10075000089587B38C6287BBC298C59822B7309141
:10076000A800432F9091A700415030F082B7821B20
:100770008917E0F34150D0F7C29A22B7315030F0D8
:1007800082B7821B8917E0F33150D0F7C29880916D
:10079000A3009091A400885F924019F01092A600E7
:1007A00008958091A5008DB98091A2008EB9109214
:1007B000A600089587B3837D87BB88B3837D88BBFC
:1007C0001DB80895CF93DF93C0E2E091A300F091AC
:1007D000A4008CEA0995E091A300F091A40083E5C0
:1007E0000995E091A300F091A40080E00995D82F2D
:1007F000E091A300F091A40080E00995D33509F4BD
:100800003AC01DB822B73091A800432F9091A7009D
:10081000415030F082B7821B8917E0F34150D0F786
:10082000C29A22B7432F415030F082B7821B8917FA
:10083000E0F34150D0F7C29822B7315030F082B780
:10084000821B8917E0F33150D0F7E091A300F091BB
:10085000A40082E0E83FF80739F0C15009F0B9CFB1
:1008600081E0DF91CF9108958091A5008DB98091AD
:10087000A2008EB9F2CF80E0DF91CF910895CF92A0
:10088000DF92EF92FF926B017C01B7DED701C601C8
:1008900081709927AA27BB27880F880F880FE091BE
:1008A000A300F091A40080620995D701C60139E048
:1008B000B695A795979587953A95D1F7E091A300BE
:1008C000F091A4000995D701C601B695A795979513
:1008D0008795E091A300F091A4000995E091A30011
:1008E000F091A40080E0FF90EF90DF90CF9009940A
:1008F000CF92DF92EF92FF920F931F93CF93DF93EC
:100900006B017C01C42FD22F78DE97018601017024
:10091000112722273327802F880F880F880FE09117
:10092000A300F091A40080640995D701C60159E0A5
:10093000B695A795979587955A95D1F7E091A3001D
:10094000F091A4000995D701C601B695A795979592
:100950008795E091A300F091A4000995E091A30090
:10096000F091A4008C2F0995DD23A9F0CF3789F0F1
:10097000D2B7CEE1C701B60182DF8F3761F482B70B
:100980008D1B8D3310F0D2B7C150C111F3CF81E070
:1009900003C08FE0B2D080E0DF91CF911F910F9123
:1009A000FF90EF90DF90CF900895CF92DF92EF927B
:1009B000FF920F931F93CF93DF931F92CDB7DEB7B4
:1009C0006B017C01498319DEE091A300F091A40042
:1009D0008CE40995D701C60179E0B695A79597955E
:1009E00087957A95D1F7E091A300F091A40009953D
:1009F000D701C601B695A79597958795E091A30075
:100A0000F091A4000995E091A300F091A40080E08A
:100A1000099549814F3FE1F002B71EE1C701B601D8
:100A20002EDF8F3F99F482B7801B8D3310F002B711
:100A300011501111F3CF81E00F90DF91CF911F91F1
:100A40000F91FF90EF90DF90CF90089580E0F4CF6A
:100A50008FE053D080E0F0CF1F93CF93DF931F92AE
:100A6000CDB7DEB7182FE091A300F091A40080EA83
:100A700099830995E091A300F091A4009981892FB1
:100A80000995E091A300F091A400812F0995E091D0
:100A9000A300F091A40080E00F90DF91CF911F910F
:100AA00009941F93CF93DF9300D0CDB7DEB7182FF3
:100AB000E091A300F091A40080EC6A8399830995EA
:100AC000E091A300F091A4009981892F0995E0910C
:100AD000A300F091A400812F0995E091A300F0916B
:100AE000A4006A81862F09958EE107D080E00F90DF
:100AF0000F90DF91CF911F910895882349F030E046
:100B000022B792B7921B9C33E0F33F5F3813F8CFC4
:100B10000895BD9ABB98C39A50E217D05A95E9F749
:100B20000895AC0188E605D0842F03D089E601D072
:100B3000852F0FD028E030E0382780FB869506D03F
:100B40002A95D1F730FB02D000D06894BB98C39AA5
:100B500016F0C398BB9AE091AA00F091AB003197D0
:100B6000F0F7C59AE6B3E3FBE091AA00F091AB0081
:100B70003197F0F7C598089520ECE7DF46F42A9501
:100B8000E1F780E02AE1E5DF2A95E9F7DECF28E00A
:100B900030E0DBDF869587F938272A95D1F7D5DF56
:100BA00027F9322772F3D1DFD0CFDB01742FB9DF01
:100BB00084E2BFDFE1DF8D937A95D1F70895DB0101
:100BC000742FAFDF83EFB5DF8DE1B3DF84E6B1DFF4
:100BD0008D91AFDF82E7ADDFCFDF8078D9F77A95EF
:100BE00089F70895CF93DF93EC018981813089F1F2
:100BF000823009F4A8C0833009F45FC08430A1F1C9
:100C0000873009F47FC0853009F4FEC0863009F4CE
:100C10009EC0883009F4D1C0893009F4FAC08A3006
:100C200009F425C18B3009F451C18C3009F461C13C
:100C30008D3009F473C18E3009F475C18F3009F419
:100C4000F9C0803109F41AC18F3709F434C180E04A
:100C50002BC09A9B54C080916300FDDC109264000D
:100C6000A99877DD80E020C080916400811110C0D8
:100C70005B8140E08A81482B662757FD6095762F7F
:100C800040936D0050936E0060936F0070937000FE
:100C90009F8180E02E81822B90937200809371005F
:100CA00082E0809373008FEF25E630E03093870079
:100CB00020938600DF91CF910895E091A300F091F9
:100CC000A4008A81099580936500E091A300F091CA
:100CD000A4008B81099580936600E091A300F091B8
:100CE000A4008C81099580936700E091A300F091A6
:100CF000A4008D8109958093680084E0D5CF85E0BC
:100D0000AADCACCF80916400811110C05B8140E00F
:100D10008A81482B662757FD6095762F40936D009A
:100D200050936E0060936F00709370009F8180E01D
:100D30002E81822B909372008093710083E08093C8
:100D400073008FEFB1CF36DDA99A80E0ADCF8091EF
:100D50006400811110C09B8180E02A81822BAA2728
:100D600097FDA095BA2F80936D0090936E00A0938D
:100D70006F00B09370003C812D81822F8F70809323
:100D80007600822F807F40E1849FC0011124830F71
:100D9000911D909375008093740020FD80937700DF
:100DA0009F8180E02E81822B90937200809371004E
:100DB00081E0809373008FEF77CF80916400811181
:100DC00010C09B8180E02A81822BAA2797FDA095E5
:100DD000BA2F80936D0090936E00A0936F00B09334
:100DE00070001092750010927400109276009F812E
:100DF00080E02E81822B909372008093710084E0BA
:100E0000809373008FEF50CFDDDC8093650081E02D
:100E10004BCF81E0809364008A819B81AC81BD814E
:100E200080936D0090936E00A0936F00B09370005C
:100E300080E03ACF9B8180E02A81822BAA2797FD10
:100E4000A095BA2F80936D0090936E00A0936F00D1
:100E5000B09370009F8180E02E81822B909372006E
:100E60008093710085E0809373008FEF1DCF8A819E
:100E7000809363001092650081E016CF9B8180E033
:100E80002A81822BAA2797FDA095BA2F80936D0007
:100E900090936E00A0936F00B09370009F8180E0EC
:100EA0002E81822B909372008093710086E0809354
:100EB00073008FEFF9CE81E0809365001092660099
:100EC000109267001092680084E0EECE9B8180E073
:100ED0002A81822B9093AB008093AA00C29ABA9A7F
:100EE00083E00BDEC298A99880E107DE12DE80E085
:100EF000DBCE80EC1EDE80E01CDE8AE0FEDDC29AE6
:100F000085E0FBDDC29885E0F8DD87B3837D87BB94
:100F100088B3837D88BBA99A80E0C6CE2DDE8093FE
:100F2000650081E0C1CE8A8104DE80E0BDCE0F93F2
:100F30001F93CF93DF93582F792F062F20917300A3
:100F4000322F3250323050F0253009F441C00FEFCB
:100F5000802FDF91CF911F910F910895662381F12A
:100F600080916D0090916E00A0916F00B091700023
:100F7000C52FD72F10E01BC06FDD888380916D00D7
:100F800090916E00A0916F00B09170000196A11D2C
:100F9000B11D80936D0090936E00A0936F00B0938D
:100FA00070001F5F2196101749F0209173002230C6
:100FB00019F7BC01CD0163DC8883E0CF083040F62F
:100FC00010927300802FDF91CF911F910F910895A0
:100FD000462F682F80916D0090916E00E6DD809124
:100FE0006D0090916E00A0916F00B0917000800F25
:100FF000911DA11DB11D80936D0090936E00A09373
:101000006F00B0937000A4CFFF920F931F93CF9304
:10101000DF93382F792F162F20917300213071F034
:10102000243061F0263009F48BC0FF24FA948F2D10
:10103000DF91CF911F910F91FF900895112309F433
:10104000ABC080916D0090916E00A0916F00B09147
:101050007000C32FD72F00E0F12C4EC020917400F8
:1010600030917500232B09F050C021E04881BC016C
:10107000CD013EDC20917100309172002150310988
:101080003093720020937100232BE1F410927300CF
:101090008091760081FF36C02091770030E080910A
:1010A0007400909175002817390761F160916D0007
:1010B00070916E0080916F0090917000488175DC96
:1010C000FF24F39480916D0090916E00A0916F00C9
:1010D000B09170000196A11DB11D80936D00909399
:1010E0006E00A0936F00B09370000F5F2196011700
:1010F00009F49DCF20917300213009F4AFCF6881AE
:10110000D0DCB8CFFF24F394DDCF20E04881BC01D0
:10111000CD01EEDB809177008150809377008111C3
:10112000A9CF60916D0070916E0080916F009091D9
:10113000700048813ADC80917400809377009ACFE8
:10114000462F682F80916D0090916E0038DD809160
:101150006D0090916E00A0916F00B0917000810FB2
:10116000911DA11DB11D80936D0090936E00A09301
:101170006F00B09370008091710090917200811B9C
:1011800091099093720080937100892B29F4109239
:101190007300FF24F3944BCFF12C49CF12BA18BA45
:1011A0008BEF81BB8FEF87BB17BA83E084BB9EEFC9
:1011B00095BB83BFA7D878947BD77AD7FDCFF89417
:0211C000FFCF5F
:0211C2005AFFD2
:00000001FF
